:020000040000FA
:0600000000000EEF00F00D
:0400080004EF00F011
:080018000CEF00F008D882741F
:1000200057D883CF05F085EC00F059D8F8D78E0E5D
:10003000C16EE10E926EDC0E936ED00E946E0F0EBA
:10004000956E000E966E880ED56E100E806E01D8DD
:1000500012000A0E036E43D80306FDE18490010EE0
:10006000F76E360EF66E08008482F5CF83FF849219
:1000700036D88482F538836E849231D80B00F552DD
:10008000F3E11200210E036E0306FEE112008490DC
:100090000800F55201E10B008482F5CF83FF8492C2
:1000A0008482F538836E8492EDDF84800B00F552F4
:1000B000F3E1120084908482EFCF83FF84928482E4
:1000C000EF38836E8492DEDF8480EC50F4E112001E
:1000D0008088040603E1FA0E046E80981200F2A4F0
:1000E000FED7F2CF02F0F29ED6CF00F0D7CF01F0CC
:1000F000660E00269E0E012201C0D7FF00C0D6FF6B
:100100000250800BF212F2941200010EF76E3E0EB6
:10011000F66EBDDF00EE0EF0E86A0532E836300913
:10012000ED6EE9500608F8E100EE06F0C00E066E2E
:100130000F6AC0DF1200333228010C060000804233
:100140005954453D20202000004890909090909078
:10015000909098989898989898989C9C9C9C9C9C17
:100160009C9C9E9E9E9E9E9E9E9E9F9F9F9F9F9FAD
:040170009F9F00004D
:020000040030CA
:08000000FFFAF6FEFFFFFBFF13
:00000001FF
